S11000008E00FFF6102EC54027F98603B7C9
S110000D102B860CB7102D8660B7103CBD7B
S110001A008825FB4D26F84F8D748D62B7CC
S10E002700A5B700A78D5AB700A6BBC8
S111003200A7B700A7CE00A8C6408D4AA700BD
S1110040085A26F818FE00A5CE00A8C640B641
S111004E00A52723A60018A7000818085A26A4
S110005CF5FC100EC34E20FD101E8608B7E3
S11100691023B5102327FBFE00A5C640A600F9
S11100778D1FBB00A7B700A7085A26F2438DC1
S111008512209CB6102E852027F985020C2728
S111009300B6102F3936B6102E848027F932AD
S10700A1B7102F3928
S9030000FC
